 clrfmodw001

 Timestamp is e1265143 (reproducible build file hash)

 Preferred load address is 0000000180000000

 Start         Length     Name                   Class
 0001:00000000 00002cc0H .text$mn                CODE
 0001:00002cc0 00000036H .text$mn$00             CODE
 0001:00002cf6 00000092H .text$x                 CODE
 0002:00000000 00000190H .idata$5                DATA
 0002:00000190 00000038H .00cfg                  DATA
 0002:000001c8 00000008H .CRT$XCA                DATA
 0002:000001d0 00000008H .CRT$XCZ                DATA
 0002:000001d8 00000008H .CRT$XIA                DATA
 0002:000001e0 00000008H .CRT$XIC                DATA
 0002:000001e8 00000008H .CRT$XIZ                DATA
 0002:000001f0 00000008H .CRT$XLA                DATA
 0002:000001f8 00000008H .CRT$XLZ                DATA
 0002:00000200 00000008H .CRT$XPA                DATA
 0002:00000208 00000008H .CRT$XPZ                DATA
 0002:00000210 00000008H .CRT$XTA                DATA
 0002:00000218 00000008H .CRT$XTZ                DATA
 0002:00000220 00000000H .gehcont$y              DATA
 0002:00000220 00000000H .gfids$y                DATA
 0002:00000220 00001ce0H .rdata                  DATA
 0002:00001f00 00000000H .rdata$CastGuardVftablesA DATA
 0002:00001f00 00000000H .rdata$CastGuardVftablesC DATA
 0002:00001f00 00000028H .rdata$T                DATA
 0002:00001f28 000000a4H .rdata$voltmd           DATA
 0002:00001fcc 0000031cH .rdata$zzzdbg           DATA
 0002:000022e8 00000008H .rtc$IAA                DATA
 0002:000022f0 00000008H .rtc$IZZ                DATA
 0002:000022f8 00000008H .rtc$TAA                DATA
 0002:00002300 00000008H .rtc$TZZ                DATA
 0002:00002308 00000004H .tls                    DATA
 0002:0000230c 00000004H .tls$                   DATA
 0002:00002310 00000008H .tls$ZZZ                DATA
 0002:00002318 000002e8H .xdata                  DATA
 0002:00002600 000004d4H .edata                  DATA
 0002:00002ad4 00000064H .idata$2                DATA
 0002:00002b38 00000018H .idata$3                DATA
 0002:00002b50 00000190H .idata$4                DATA
 0002:00002ce0 00000414H .idata$6                DATA
 0003:00000000 00000140H .data                   DATA
 0003:00000140 0001b388H .bss                    DATA
 0004:00000000 00000384H .pdata                  DATA

  Address         Publics by Value              Rva+Base               Lib:Object

 0000:00000000       __AbsoluteZero             0000000000000000     <absolute>
 0000:00000000       ___safe_se_handler_count   0000000000000000     <absolute>
 0000:00000000       ___safe_se_handler_table   0000000000000000     <absolute>
 0000:00000000       __arm64x_extra_rfe_table   0000000000000000     <absolute>
 0000:00000000       __arm64x_extra_rfe_table_size 0000000000000000     <absolute>
 0000:00000000       __arm64x_native_entrypoint 0000000000000000     <absolute>
 0000:00000000       __arm64x_redirection_metadata 0000000000000000     <absolute>
 0000:00000000       __arm64x_redirection_metadata_count 0000000000000000     <absolute>
 0000:00000000       __dynamic_value_reloc_table 0000000000000000     <absolute>
 0000:00000000       __enclave_config           0000000000000000     <absolute>
 0000:00000000       __guard_check_icall_a64n_fptr 0000000000000000     <absolute>
 0000:00000000       __guard_eh_cont_count      0000000000000000     <absolute>
 0000:00000000       __guard_eh_cont_table      0000000000000000     <absolute>
 0000:00000000       __guard_fids_count         0000000000000000     <absolute>
 0000:00000000       __guard_fids_table         0000000000000000     <absolute>
 0000:00000000       __guard_iat_count          0000000000000000     <absolute>
 0000:00000000       __guard_iat_table          0000000000000000     <absolute>
 0000:00000000       __guard_longjmp_count      0000000000000000     <absolute>
 0000:00000000       __guard_longjmp_table      0000000000000000     <absolute>
 0000:00000000       __hybrid_auxiliary_iat     0000000000000000     <absolute>
 0000:00000000       __hybrid_auxiliary_iat_copy 0000000000000000     <absolute>
 0000:00000000       __hybrid_code_map          0000000000000000     <absolute>
 0000:00000000       __hybrid_code_map_count    0000000000000000     <absolute>
 0000:00000000       __x64_code_ranges_to_entry_points 0000000000000000     <absolute>
 0000:00000000       __x64_code_ranges_to_entry_points_count 0000000000000000     <absolute>
 0000:00000100       __guard_flags              0000000000000100     <absolute>
 0000:00000000       __ImageBase                0000000180000000     <linker-defined>
 0001:00000000       ?NewObject@JNIEnv_@@QEAAPEAV_jobject@@PEAV_jclass@@PEAU_jmethodID@@ZZ 0000000180001000 f i libclrfmodw001.obj
 0001:00000028       ?SetEventNotificationMode@_jvmtiEnv@@QEAA?AW4jvmtiError@@W4jvmtiEventMode@@W4jvmtiEvent@@PEAV_jobject@@ZZ 0000000180001028 f i libclrfmodw001.obj
 0001:00000034       ?TranslateError@@YAPEBDW4jvmtiError@@@Z 0000000180001034 f   libclrfmodw001.obj
 0001:000002ec       ?nsk_jni_check_exception@@YAHPEAUJNIEnv_@@QEBDH@Z 00000001800012ec f   libclrfmodw001.obj
 0001:00000430       ?nsk_jni_lverify@@YAHHPEAUJNIEnv_@@HQEBDH1ZZ 0000000180001430 f   libclrfmodw001.obj
 0001:000004d0       Agent_Initialize           00000001800014d0 f   libclrfmodw001.obj
 0001:00000648       Agent_OnAttach             0000000180001648 f   libclrfmodw001.obj
 0001:00000648       Agent_OnLoad               0000000180001648 f   libclrfmodw001.obj
 0001:00000650       FieldModification          0000000180001650 f   libclrfmodw001.obj
 0001:00000660       Java_nsk_jvmti_ClearFieldModificationWatch_clrfmodw001_check 0000000180001660 f   libclrfmodw001.obj
 0001:000006ec       Java_nsk_jvmti_ClearFieldModificationWatch_clrfmodw001_clearWatch 00000001800016ec f   libclrfmodw001.obj
 0001:000006f8       Java_nsk_jvmti_ClearFieldModificationWatch_clrfmodw001_getRes 00000001800016f8 f   libclrfmodw001.obj
 0001:00000700       Java_nsk_jvmti_ClearFieldModificationWatch_clrfmodw001_setWatch 0000000180001700 f   libclrfmodw001.obj
 0001:0000070c       Java_nsk_jvmti_ClearFieldModificationWatch_clrfmodw001_touchfld0 000000018000170c f   libclrfmodw001.obj
 0001:00000724       Java_nsk_jvmti_unit_FollowReferences_FollowRefObjects_addRefToVerify 0000000180001724 f   libclrfmodw001.obj
 0001:000008fc       Java_nsk_jvmti_unit_FollowReferences_FollowRefObjects_getTag 00000001800018fc f   libclrfmodw001.obj
 0001:000009bc       Java_nsk_jvmti_unit_FollowReferences_FollowRefObjects_resetRefsToVerify 00000001800019bc f   libclrfmodw001.obj
 0001:000009c4       Java_nsk_jvmti_unit_FollowReferences_FollowRefObjects_resetTags 00000001800019c4 f   libclrfmodw001.obj
 0001:00000a08       Java_nsk_jvmti_unit_FollowReferences_FollowRefObjects_setTag 0000000180001a08 f   libclrfmodw001.obj
 0001:00000c60       Java_nsk_share_jvmti_ArgumentHandler_getAgentOptionsString 0000000180001c60 f   libclrfmodw001.obj
 0001:00000d10       Java_nsk_share_jvmti_DebugeeClass_checkStatus 0000000180001d10 f   libclrfmodw001.obj
 0001:00000d98       Java_nsk_share_jvmti_DebugeeClass_resetAgentData 0000000180001d98 f   libclrfmodw001.obj
 0001:00000df8       Java_nsk_share_jvmti_RedefineAgent_agentStatus 0000000180001df8 f   libclrfmodw001.obj
 0001:00000e04       Java_nsk_share_jvmti_RedefineAgent_isRedefined 0000000180001e04 f   libclrfmodw001.obj
 0001:00000e10       Java_nsk_share_jvmti_RedefineAgent_redefineAttempted 0000000180001e10 f   libclrfmodw001.obj
 0001:00000e1c       MA_checkStatus             0000000180001e1c f   libclrfmodw001.obj
 0001:00000ec0       __local_stdio_printf_options 0000000180001ec0 f i libclrfmodw001.obj
 0001:000010a0       exitOnError                00000001800020a0 f   libclrfmodw001.obj
 0001:00001154       fprintf                    0000000180002154 f i libclrfmodw001.obj
 0001:00001198       nsk_jvmti_lverify          0000000180002198 f   libclrfmodw001.obj
 0001:00001288       nsk_jvmti_resetAgentData   0000000180002288 f   libclrfmodw001.obj
 0001:00001308       nsk_jvmti_setFailStatus    0000000180002308 f   libclrfmodw001.obj
 0001:00001344       nsk_lcomplain              0000000180002344 f   libclrfmodw001.obj
 0001:00001364       nsk_ldisplay               0000000180002364 f   libclrfmodw001.obj
 0001:00001384       nsk_ltrace                 0000000180002384 f   libclrfmodw001.obj
 0001:000013a4       nsk_lvcomplain             00000001800023a4 f   libclrfmodw001.obj
 0001:0000155c       nsk_lvdisplay              000000018000255c f   libclrfmodw001.obj
 0001:000015a8       nsk_lverify                00000001800025a8 f   libclrfmodw001.obj
 0001:00001604       nsk_lvtrace                0000000180002604 f   libclrfmodw001.obj
 0001:00001664       nsk_printf                 0000000180002664 f   libclrfmodw001.obj
 0001:0000168c       nsk_vprintf                000000018000268c f   libclrfmodw001.obj
 0001:00001740       printf                     0000000180002740 f i libclrfmodw001.obj
 0001:00001ad0       switchWatch                0000000180002ad0 f   libclrfmodw001.obj
 0001:00001d94       __raise_securityfailure    0000000180002d94 f   MSVCRT:gs_report.obj
 0001:00001dc8       __report_gsfailure         0000000180002dc8 f   MSVCRT:gs_report.obj
 0001:00002008       __GSHandlerCheck           0000000180003008 f   MSVCRT:gshandler.obj
 0001:00002028       __GSHandlerCheckCommon     0000000180003028 f   MSVCRT:gshandler.obj
 0001:000020a0       __security_check_cookie    00000001800030a0 f   MSVCRT:amdsecgs.obj
 0001:000023e0       _DllMainCRTStartup         00000001800033e0 f   MSVCRT:dll_dllmain.obj
 0001:00002420       __scrt_acquire_startup_lock 0000000180003420 f   MSVCRT:utility.obj
 0001:0000245c       __scrt_dllmain_after_initialize_c 000000018000345c f   MSVCRT:utility.obj
 0001:00002490       __scrt_dllmain_before_initialize_c 0000000180003490 f   MSVCRT:utility.obj
 0001:000024a8       __scrt_dllmain_crt_thread_attach 00000001800034a8 f   MSVCRT:utility.obj
 0001:000024d0       __scrt_dllmain_crt_thread_detach 00000001800034d0 f   MSVCRT:utility.obj
 0001:000024e8       __scrt_dllmain_exception_filter 00000001800034e8 f   MSVCRT:utility.obj
 0001:00002548       __scrt_dllmain_uninitialize_c 0000000180003548 f   MSVCRT:utility.obj
 0001:00002578       __scrt_dllmain_uninitialize_critical 0000000180003578 f   MSVCRT:utility.obj
 0001:0000258c       __scrt_initialize_crt      000000018000358c f   MSVCRT:utility.obj
 0001:000025d8       __scrt_initialize_onexit_tables 00000001800035d8 f   MSVCRT:utility.obj
 0001:00002664       __scrt_is_nonwritable_in_current_image 0000000180003664 f   MSVCRT:utility.obj
 0001:000026fc       __scrt_release_startup_lock 00000001800036fc f   MSVCRT:utility.obj
 0001:00002720       __scrt_uninitialize_crt    0000000180003720 f   MSVCRT:utility.obj
 0001:0000274c       _onexit                    000000018000374c f   MSVCRT:utility.obj
 0001:00002788       atexit                     0000000180003788 f   MSVCRT:utility.obj
 0001:000027a0       __crt_debugger_hook        00000001800037a0 f   MSVCRT:utility_desktop.obj
 0001:000027a8       __scrt_fastfail            00000001800037a8 f   MSVCRT:utility_desktop.obj
 0001:000028f4       _guard_check_icall_nop     00000001800038f4 f i MSVCRT:guard_support.obj
 0001:000028f8       __security_init_cookie     00000001800038f8 f   MSVCRT:gs_support.obj
 0001:000029a4       DllMain                    00000001800039a4 f   MSVCRT:dll_dllmain_stub.obj
 0001:000029c8       ?__scrt_initialize_type_info@@YAXXZ 00000001800039c8 f   MSVCRT:tncleanup.obj
 0001:000029d8       ?__scrt_uninitialize_type_info@@YAXXZ 00000001800039d8 f   MSVCRT:tncleanup.obj
 0001:000029e4       __local_stdio_scanf_options 00000001800039e4 f i MSVCRT:default_local_stdio_options.obj
 0001:000029ec       __scrt_initialize_default_local_stdio_options 00000001800039ec f   MSVCRT:default_local_stdio_options.obj
 0001:00002a08       __scrt_get_dyn_tls_init_callback 0000000180003a08 f   MSVCRT:dyn_tls_init.obj
 0001:00002a10       _RTC_Initialize            0000000180003a10 f   MSVCRT:initsect.obj
 0001:00002a4c       _RTC_Terminate             0000000180003a4c f   MSVCRT:initsect.obj
 0001:00002a88       __isa_available_init       0000000180003a88 f   MSVCRT:cpu_disp.obj
 0001:00002c34       _get_startup_argv_mode     0000000180003c34 f   MSVCRT:argv_mode.obj
 0001:00002c3c       __scrt_is_ucrt_dll_in_use  0000000180003c3c f   MSVCRT:ucrt_detection.obj
 0001:00002c50       memcpy                     0000000180003c50 f   vcruntime:VCRUNTIME140.dll
 0001:00002c56       memset                     0000000180003c56 f   vcruntime:VCRUNTIME140.dll
 0001:00002c5c       strchr                     0000000180003c5c f   vcruntime:VCRUNTIME140.dll
 0001:00002c62       __C_specific_handler       0000000180003c62 f   vcruntime:VCRUNTIME140.dll
 0001:00002c68       __std_type_info_destroy_list 0000000180003c68 f   vcruntime:VCRUNTIME140.dll
 0001:00002c6e       strlen                     0000000180003c6e f   ucrt:api-ms-win-crt-string-l1-1-0.dll
 0001:00002c74       _initterm                  0000000180003c74 f   ucrt:api-ms-win-crt-runtime-l1-1-0.dll
 0001:00002c7a       _initterm_e                0000000180003c7a f   ucrt:api-ms-win-crt-runtime-l1-1-0.dll
 0001:00002c80       _seh_filter_dll            0000000180003c80 f   ucrt:api-ms-win-crt-runtime-l1-1-0.dll
 0001:00002c86       _configure_narrow_argv     0000000180003c86 f   ucrt:api-ms-win-crt-runtime-l1-1-0.dll
 0001:00002c8c       _initialize_narrow_environment 0000000180003c8c f   ucrt:api-ms-win-crt-runtime-l1-1-0.dll
 0001:00002c92       _initialize_onexit_table   0000000180003c92 f   ucrt:api-ms-win-crt-runtime-l1-1-0.dll
 0001:00002c98       _register_onexit_function  0000000180003c98 f   ucrt:api-ms-win-crt-runtime-l1-1-0.dll
 0001:00002c9e       _execute_onexit_table      0000000180003c9e f   ucrt:api-ms-win-crt-runtime-l1-1-0.dll
 0001:00002ca4       _crt_atexit                0000000180003ca4 f   ucrt:api-ms-win-crt-runtime-l1-1-0.dll
 0001:00002caa       _cexit                     0000000180003caa f   ucrt:api-ms-win-crt-runtime-l1-1-0.dll
 0001:00002cb0       __acrt_initialize          0000000180003cb0 f   MSVCRT:ucrt_stubs.obj
 0001:00002cb0       __acrt_thread_attach       0000000180003cb0 f   MSVCRT:ucrt_stubs.obj
 0001:00002cb0       __acrt_thread_detach       0000000180003cb0 f   MSVCRT:ucrt_stubs.obj
 0001:00002cb0       __acrt_uninitialize        0000000180003cb0 f   MSVCRT:ucrt_stubs.obj
 0001:00002cb0       __acrt_uninitialize_critical 0000000180003cb0 f   MSVCRT:ucrt_stubs.obj
 0001:00002cb0       __scrt_stub_for_acrt_initialize 0000000180003cb0 f   MSVCRT:ucrt_stubs.obj
 0001:00002cb0       __scrt_stub_for_acrt_thread_attach 0000000180003cb0 f   MSVCRT:ucrt_stubs.obj
 0001:00002cb0       __scrt_stub_for_acrt_thread_detach 0000000180003cb0 f   MSVCRT:ucrt_stubs.obj
 0001:00002cb0       __scrt_stub_for_acrt_uninitialize 0000000180003cb0 f   MSVCRT:ucrt_stubs.obj
 0001:00002cb0       __scrt_stub_for_acrt_uninitialize_critical 0000000180003cb0 f   MSVCRT:ucrt_stubs.obj
 0001:00002cb0       __vcrt_initialize          0000000180003cb0 f   MSVCRT:ucrt_stubs.obj
 0001:00002cb0       __vcrt_thread_attach       0000000180003cb0 f   MSVCRT:ucrt_stubs.obj
 0001:00002cb0       __vcrt_thread_detach       0000000180003cb0 f   MSVCRT:ucrt_stubs.obj
 0001:00002cb0       __vcrt_uninitialize        0000000180003cb0 f   MSVCRT:ucrt_stubs.obj
 0001:00002cb0       __vcrt_uninitialize_critical 0000000180003cb0 f   MSVCRT:ucrt_stubs.obj
 0001:00002cb4       __scrt_stub_for_is_c_termination_complete 0000000180003cb4 f   MSVCRT:ucrt_stubs.obj
 0001:00002cb4       _is_c_termination_complete 0000000180003cb4 f   MSVCRT:ucrt_stubs.obj
 0001:00002cd0       _guard_dispatch_icall_nop  0000000180003cd0 f   MSVCRT:guard_dispatch.obj
 0001:00002cf0       _guard_xfg_dispatch_icall_nop 0000000180003cf0 f   MSVCRT:guard_xfg_dispatch.obj
 0002:00000000       __imp_RtlCaptureContext    0000000180004000     kernel32:KERNEL32.dll
 0002:00000008       __imp_RtlLookupFunctionEntry 0000000180004008     kernel32:KERNEL32.dll
 0002:00000010       __imp_RtlVirtualUnwind     0000000180004010     kernel32:KERNEL32.dll
 0002:00000018       __imp_UnhandledExceptionFilter 0000000180004018     kernel32:KERNEL32.dll
 0002:00000020       __imp_SetUnhandledExceptionFilter 0000000180004020     kernel32:KERNEL32.dll
 0002:00000028       __imp_GetCurrentProcess    0000000180004028     kernel32:KERNEL32.dll
 0002:00000030       __imp_TerminateProcess     0000000180004030     kernel32:KERNEL32.dll
 0002:00000038       __imp_IsProcessorFeaturePresent 0000000180004038     kernel32:KERNEL32.dll
 0002:00000040       __imp_CloseHandle          0000000180004040     kernel32:KERNEL32.dll
 0002:00000048       __imp_InitializeCriticalSectionAndSpinCount 0000000180004048     kernel32:KERNEL32.dll
 0002:00000050       __imp_DeleteCriticalSection 0000000180004050     kernel32:KERNEL32.dll
 0002:00000058       __imp_CreateEventW         0000000180004058     kernel32:KERNEL32.dll
 0002:00000060       __imp_GetModuleHandleW     0000000180004060     kernel32:KERNEL32.dll
 0002:00000068       __imp_GetProcAddress       0000000180004068     kernel32:KERNEL32.dll
 0002:00000070       __imp_IsDebuggerPresent    0000000180004070     kernel32:KERNEL32.dll
 0002:00000078       __imp_QueryPerformanceCounter 0000000180004078     kernel32:KERNEL32.dll
 0002:00000080       __imp_GetCurrentProcessId  0000000180004080     kernel32:KERNEL32.dll
 0002:00000088       __imp_GetCurrentThreadId   0000000180004088     kernel32:KERNEL32.dll
 0002:00000090       __imp_GetSystemTimeAsFileTime 0000000180004090     kernel32:KERNEL32.dll
 0002:00000098       __imp_DisableThreadLibraryCalls 0000000180004098     kernel32:KERNEL32.dll
 0002:000000a0       __imp_InitializeSListHead  00000001800040a0     kernel32:KERNEL32.dll
 0002:000000a8       \177KERNEL32_NULL_THUNK_DATA 00000001800040a8     kernel32:KERNEL32.dll
 0002:000000b0       __imp_memcpy               00000001800040b0     vcruntime:VCRUNTIME140.dll
 0002:000000b8       __imp_memset               00000001800040b8     vcruntime:VCRUNTIME140.dll
 0002:000000c0       __imp_strchr               00000001800040c0     vcruntime:VCRUNTIME140.dll
 0002:000000c8       __imp___C_specific_handler 00000001800040c8     vcruntime:VCRUNTIME140.dll
 0002:000000d0       __imp___std_type_info_destroy_list 00000001800040d0     vcruntime:VCRUNTIME140.dll
 0002:000000d8       \177VCRUNTIME140_NULL_THUNK_DATA 00000001800040d8     vcruntime:VCRUNTIME140.dll
 0002:000000e0       __imp__errno               00000001800040e0     ucrt:api-ms-win-crt-runtime-l1-1-0.dll
 0002:000000e8       __imp_exit                 00000001800040e8     ucrt:api-ms-win-crt-runtime-l1-1-0.dll
 0002:000000f0       __imp__cexit               00000001800040f0     ucrt:api-ms-win-crt-runtime-l1-1-0.dll
 0002:000000f8       __imp__crt_atexit          00000001800040f8     ucrt:api-ms-win-crt-runtime-l1-1-0.dll
 0002:00000100       __imp__execute_onexit_table 0000000180004100     ucrt:api-ms-win-crt-runtime-l1-1-0.dll
 0002:00000108       __imp__register_onexit_function 0000000180004108     ucrt:api-ms-win-crt-runtime-l1-1-0.dll
 0002:00000110       __imp__initialize_onexit_table 0000000180004110     ucrt:api-ms-win-crt-runtime-l1-1-0.dll
 0002:00000118       __imp__initialize_narrow_environment 0000000180004118     ucrt:api-ms-win-crt-runtime-l1-1-0.dll
 0002:00000120       __imp__configure_narrow_argv 0000000180004120     ucrt:api-ms-win-crt-runtime-l1-1-0.dll
 0002:00000128       __imp__seh_filter_dll      0000000180004128     ucrt:api-ms-win-crt-runtime-l1-1-0.dll
 0002:00000130       __imp__initterm_e          0000000180004130     ucrt:api-ms-win-crt-runtime-l1-1-0.dll
 0002:00000138       __imp__initterm            0000000180004138     ucrt:api-ms-win-crt-runtime-l1-1-0.dll
 0002:00000140       \177api-ms-win-crt-runtime-l1-1-0_NULL_THUNK_DATA 0000000180004140     ucrt:api-ms-win-crt-runtime-l1-1-0.dll
 0002:00000148       __imp___acrt_iob_func      0000000180004148     ucrt:api-ms-win-crt-stdio-l1-1-0.dll
 0002:00000150       __imp_fflush               0000000180004150     ucrt:api-ms-win-crt-stdio-l1-1-0.dll
 0002:00000158       __imp___stdio_common_vsprintf 0000000180004158     ucrt:api-ms-win-crt-stdio-l1-1-0.dll
 0002:00000160       __imp___stdio_common_vfprintf 0000000180004160     ucrt:api-ms-win-crt-stdio-l1-1-0.dll
 0002:00000168       \177api-ms-win-crt-stdio-l1-1-0_NULL_THUNK_DATA 0000000180004168     ucrt:api-ms-win-crt-stdio-l1-1-0.dll
 0002:00000170       __imp__strdup              0000000180004170     ucrt:api-ms-win-crt-string-l1-1-0.dll
 0002:00000170       __imp_strdup               0000000180004170     ucrt:api-ms-win-crt-string-l1-1-0.dll
 0002:00000178       __imp_strlen               0000000180004178     ucrt:api-ms-win-crt-string-l1-1-0.dll
 0002:00000180       __imp_strncpy              0000000180004180     ucrt:api-ms-win-crt-string-l1-1-0.dll
 0002:00000188       \177api-ms-win-crt-string-l1-1-0_NULL_THUNK_DATA 0000000180004188     ucrt:api-ms-win-crt-string-l1-1-0.dll
 0002:00000190       __guard_check_icall_fptr   0000000180004190     MSVCRT:guard_support.obj
 0002:00000198       __guard_xfg_check_icall_fptr 0000000180004198     MSVCRT:guard_support.obj
 0002:000001a0       __guard_dispatch_icall_fptr 00000001800041a0     MSVCRT:guard_support.obj
 0002:000001a8       __guard_xfg_dispatch_icall_fptr 00000001800041a8     MSVCRT:guard_support.obj
 0002:000001b0       __guard_xfg_table_dispatch_icall_fptr 00000001800041b0     MSVCRT:guard_support.obj
 0002:000001b8       __castguard_check_failure_os_handled_fptr 00000001800041b8     MSVCRT:guard_support.obj
 0002:000001c0       __guard_memcpy_fptr        00000001800041c0     vcruntime:softmemtag.obj
 0002:000001c8       __xc_a                     00000001800041c8     MSVCRT:initializers.obj
 0002:000001d0       __xc_z                     00000001800041d0     MSVCRT:initializers.obj
 0002:000001d8       __xi_a                     00000001800041d8     MSVCRT:initializers.obj
 0002:000001e8       __xi_z                     00000001800041e8     MSVCRT:initializers.obj
 0002:000001f0       __xl_a                     00000001800041f0     MSVCRT:tlssup.obj
 0002:000001f8       __xl_z                     00000001800041f8     MSVCRT:tlssup.obj
 0002:00000200       __xp_a                     0000000180004200     MSVCRT:initializers.obj
 0002:00000208       __xp_z                     0000000180004208     MSVCRT:initializers.obj
 0002:00000210       __xt_a                     0000000180004210     MSVCRT:initializers.obj
 0002:00000218       __xt_z                     0000000180004218     MSVCRT:initializers.obj
 0002:00000220       g_refKindStr               0000000180004220     libclrfmodw001.obj
 0002:000003d0       ??_C@_09BPLDFGCI@unknown_0@ 00000001800043d0     libclrfmodw001.obj
 0002:000003e0       ??_C@_0BL@FPNMECJD@JVMTI_HEAP_REFERENCE_CLASS@ 00000001800043e0     libclrfmodw001.obj
 0002:00000400       ??_C@_0BL@FKGKKLNM@JVMTI_HEAP_REFERENCE_FIELD@ 0000000180004400     libclrfmodw001.obj
 0002:00000420       ??_C@_0CD@CAEHCFJF@JVMTI_HEAP_REFERENCE_ARRAY_ELEM@ 0000000180004420     libclrfmodw001.obj
 0002:00000448       ??_C@_0CC@DNEBMCNK@JVMTI_HEAP_REFERENCE_CLASS_LOAD@ 0000000180004448     libclrfmodw001.obj
 0002:00000470       ??_C@_0BN@CJMIPEBB@JVMTI_HEAP_REFERENCE_SIGNERS@ 0000000180004470     libclrfmodw001.obj
 0002:00000490       ??_C@_0CH@HBOIDPEB@JVMTI_HEAP_REFERENCE_PROTECTION@ 0000000180004490     libclrfmodw001.obj
 0002:000004b8       ??_C@_0BP@MDKGDGKL@JVMTI_HEAP_REFERENCE_INTERFACE@ 00000001800044b8     libclrfmodw001.obj
 0002:000004d8       ??_C@_0CC@JJMIHNJH@JVMTI_HEAP_REFERENCE_STATIC_FIE@ 00000001800044d8     libclrfmodw001.obj
 0002:00000500       ??_C@_0CD@IDHEEGID@JVMTI_HEAP_REFERENCE_CONSTANT_P@ 0000000180004500     libclrfmodw001.obj
 0002:00000528       ??_C@_0CA@EFFCHNG@JVMTI_HEAP_REFERENCE_SUPERCLASS@ 0000000180004528     libclrfmodw001.obj
 0002:00000548       ??_C@_0L@PCDFHGCJ@unknown_11@ 0000000180004548     libclrfmodw001.obj
 0002:00000558       ??_C@_0L@NJBICFOK@unknown_12@ 0000000180004558     libclrfmodw001.obj
 0002:00000568       ??_C@_0L@MAADBEKL@unknown_13@ 0000000180004568     libclrfmodw001.obj
 0002:00000578       ??_C@_0L@IPECICGM@unknown_14@ 0000000180004578     libclrfmodw001.obj
 0002:00000588       ??_C@_0L@JGFJLDCN@unknown_15@ 0000000180004588     libclrfmodw001.obj
 0002:00000598       ??_C@_0L@LNHEOAOO@unknown_16@ 0000000180004598     libclrfmodw001.obj
 0002:000005a8       ??_C@_0L@KEGPNBKP@unknown_17@ 00000001800045a8     libclrfmodw001.obj
 0002:000005b8       ??_C@_0L@CDPHMNGA@unknown_18@ 00000001800045b8     libclrfmodw001.obj
 0002:000005c8       ??_C@_0L@DKOMPMCB@unknown_19@ 00000001800045c8     libclrfmodw001.obj
 0002:000005d8       ??_C@_0L@OJGIPJDB@unknown_20@ 00000001800045d8     libclrfmodw001.obj
 0002:000005e8       ??_C@_0CA@KAOFNDEM@JVMTI_HEAP_REFERENCE_JNI_GLOBAL@ 00000001800045e8     libclrfmodw001.obj
 0002:00000608       ??_C@_0CC@HPFAJBK@JVMTI_HEAP_REFERENCE_SYSTEM_CLA@ 0000000180004608     libclrfmodw001.obj
 0002:00000630       ??_C@_0BN@FDEGFOHC@JVMTI_HEAP_REFERENCE_MONITOR@ 0000000180004630     libclrfmodw001.obj
 0002:00000650       ??_C@_0CB@HKIBCMAJ@JVMTI_HEAP_REFERENCE_STACK_LOCA@ 0000000180004650     libclrfmodw001.obj
 0002:00000678       ??_C@_0BP@EAACMMOE@JVMTI_HEAP_REFERENCE_JNI_LOCAL@ 0000000180004678     libclrfmodw001.obj
 0002:00000698       ??_C@_0BM@IJDEOGOE@JVMTI_HEAP_REFERENCE_THREAD@ 0000000180004698     libclrfmodw001.obj
 0002:000006b8       ??_C@_0BL@EDGPPKC@JVMTI_HEAP_REFERENCE_OTHER@ 00000001800046b8     libclrfmodw001.obj
 0002:000006d4       ??_C@_04BCJPDBDA@Code@     00000001800046d4     libclrfmodw001.obj
 0002:000006e0       ??_C@_0BA@OCLMCFKC@LineNumberTable@ 00000001800046e0     libclrfmodw001.obj
 0002:000006f0       ??_C@_0BD@CPAEPILC@LocalVariableTable@ 00000001800046f0     libclrfmodw001.obj
 0002:00000708       ??_C@_0BH@NMBDNHBD@LocalVariableTypeTable@ 0000000180004708     libclrfmodw001.obj
 0002:00000720       ??_C@_0O@HIHEEDNJ@StackMapTable@ 0000000180004720     libclrfmodw001.obj
 0002:00000730       ??_C@_0DC@FLMFLDKG@nsk?1jvmti?1ClearFieldModificatio@ 0000000180004730     libclrfmodw001.obj
 0002:00000764       ??_C@_04MOMHJHLL@fld0@     0000000180004764     libclrfmodw001.obj
 0002:0000076c       ??_C@_01JPJNBJEM@I@        000000018000476c     libclrfmodw001.obj
 0002:00000770       ??_C@_04NHNMKGPK@fld1@     0000000180004770     libclrfmodw001.obj
 0002:00000778       ??_C@_04PMPBPFDJ@fld2@     0000000180004778     libclrfmodw001.obj
 0002:00000780       ??_C@_0DF@GINKDFB@Lnsk?1jvmti?1ClearFieldModificati@ 0000000180004780     libclrfmodw001.obj
 0002:000007b8       ??_C@_0DD@EDAIJJII@nsk?1jvmti?1ClearFieldModificatio@ 00000001800047b8     libclrfmodw001.obj
 0002:000007ec       ??_C@_04OFOKMEHI@fld3@     00000001800047ec     libclrfmodw001.obj
 0002:000007f4       ??_C@_02EBOMBDPA@?$FLI@    00000001800047f4     libclrfmodw001.obj
 0002:000007f8       ??_C@_0DD@GICFMKEL@nsk?1jvmti?1ClearFieldModificatio@ 00000001800047f8     libclrfmodw001.obj
 0002:0000082c       ??_C@_04KKKLFCLP@fld4@     000000018000482c     libclrfmodw001.obj
 0002:00000834       ??_C@_01BIAFAFID@F@        0000000180004834     libclrfmodw001.obj
 0002:00000838       ??_C@_0L@HCDIAMJG@?9?5?$CFs?0?5?$CFd?3?5@ 0000000180004838     libclrfmodw001.obj
 0002:00000850       ??_C@_0JI@HLPECLFI@?$CD?5?4?4?4?6?$CD?5ERROR?3?5too?5many?5complai@ 0000000180004850     libclrfmodw001.obj
 0002:000008f0       ??_C@_0ED@JNEKCCOB@The?5following?5fake?5exception?5st@ 00000001800048f0     libclrfmodw001.obj
 0002:00000938       ??_C@_0CN@FCNMDFBH@nsk?4share?4Fake_Exception_for_RU@ 0000000180004938     libclrfmodw001.obj
 0002:00000968       ??_C@_08PGFFNAEI@?$CI?$CFs?3?$CFd?$CJ?5@ 0000000180004968     libclrfmodw001.obj
 0002:00000978       ??_C@_0DP@IENMAEGI@s?2test?2hotspot?2jtreg?2vmTestbase@ 0000000180004978     libclrfmodw001.obj
 0002:000009b8       ??_C@_0BL@NDJLFFJB@?7at?5nsk_lvcomplain?$CI?$CFs?3?$CFd?$CJ?6@ 00000001800049b8     libclrfmodw001.obj
 0002:000009d8       ??_C@_0BC@JOOKAFKF@?$CD?5ERROR?3?5?$CFs?0?5?$CFd?3?5@ 00000001800049d8     libclrfmodw001.obj
 0002:000009f0       ??_C@_09KJEAHMEH@?$CD?5ERROR?3?5@ 00000001800049f0     libclrfmodw001.obj
 0002:000009fc       ??_C@_02GPIOPFAK@?$DO?$DO@ 00000001800049fc     libclrfmodw001.obj
 0002:00000a00       ??_C@_02FODMEDOG@?$DM?$DM@ 0000000180004a00     libclrfmodw001.obj
 0002:00000a04       ??_C@_02DJGKEECL@?4?4@     0000000180004a04     libclrfmodw001.obj
 0002:00000a08       ??_C@_0O@CJPGJOAF@?9?5?$CFs?0?5?$CFd?3?5?$CFs?5@ 0000000180004a08     libclrfmodw001.obj
 0002:00000a18       ??_C@_0CB@IAKPDOIC@?$CD?5?5?5verified?5assertion?5is?5FALSE@ 0000000180004a18     libclrfmodw001.obj
 0002:00000a40       ??_C@_0CO@LGONDEPD@stdout?3?5fflush?5failed?5?9?5err?$DN?$CFd?5@ 0000000180004a40     libclrfmodw001.obj
 0002:00000a70       ??_C@_0CO@KBGKJPBD@stderr?3?5fflush?5failed?5?9?5err?$DN?$CFd?5@ 0000000180004a70     libclrfmodw001.obj
 0002:00000aa0       ??_C@_0BB@JCNMKLLK@JVMTI_ERROR_NONE@ 0000000180004aa0     libclrfmodw001.obj
 0002:00000ab8       ??_C@_0BL@LDIMKLPH@JVMTI_ERROR_INVALID_THREAD@ 0000000180004ab8     libclrfmodw001.obj
 0002:00000ad8       ??_C@_0CB@PJFPAIKJ@JVMTI_ERROR_INVALID_THREAD_GROU@ 0000000180004ad8     libclrfmodw001.obj
 0002:00000b00       ??_C@_0BN@LLMKHMNF@JVMTI_ERROR_INVALID_PRIORITY@ 0000000180004b00     libclrfmodw001.obj
 0002:00000b20       ??_C@_0CB@MBOFKAGB@JVMTI_ERROR_THREAD_NOT_SUSPENDE@ 0000000180004b20     libclrfmodw001.obj
 0002:00000b48       ??_C@_0BN@FABOLPBI@JVMTI_ERROR_THREAD_SUSPENDED@ 0000000180004b48     libclrfmodw001.obj
 0002:00000b68       ??_C@_0BN@FDGNOBJM@JVMTI_ERROR_THREAD_NOT_ALIVE@ 0000000180004b68     libclrfmodw001.obj
 0002:00000b88       ??_C@_0BL@GOBIFKNJ@JVMTI_ERROR_INVALID_OBJECT@ 0000000180004b88     libclrfmodw001.obj
 0002:00000ba8       ??_C@_0BK@FCMAJPPC@JVMTI_ERROR_INVALID_CLASS@ 0000000180004ba8     libclrfmodw001.obj
 0002:00000bc8       ??_C@_0BP@IKLLBKEB@JVMTI_ERROR_CLASS_NOT_PREPARED@ 0000000180004bc8     libclrfmodw001.obj
 0002:00000be8       ??_C@_0BN@KLPPLKG@JVMTI_ERROR_INVALID_METHODID@ 0000000180004be8     libclrfmodw001.obj
 0002:00000c08       ??_C@_0BN@BCEKOKND@JVMTI_ERROR_INVALID_LOCATION@ 0000000180004c08     libclrfmodw001.obj
 0002:00000c28       ??_C@_0BM@DFDGPME@JVMTI_ERROR_INVALID_FIELDID@ 0000000180004c28     libclrfmodw001.obj
 0002:00000c48       ??_C@_0BL@NELIEPEC@JVMTI_ERROR_NO_MORE_FRAMES@ 0000000180004c48     libclrfmodw001.obj
 0002:00000c68       ??_C@_0BJ@BDBECFDM@JVMTI_ERROR_OPAQUE_FRAME@ 0000000180004c68     libclrfmodw001.obj
 0002:00000c88       ??_C@_0BK@MIIFNLOB@JVMTI_ERROR_TYPE_MISMATCH@ 0000000180004c88     libclrfmodw001.obj
 0002:00000ca8       ??_C@_0BJ@HPCAOILC@JVMTI_ERROR_INVALID_SLOT@ 0000000180004ca8     libclrfmodw001.obj
 0002:00000cc8       ??_C@_0BG@CHILOPNI@JVMTI_ERROR_DUPLICATE@ 0000000180004cc8     libclrfmodw001.obj
 0002:00000ce0       ??_C@_0BG@DIEMLHKM@JVMTI_ERROR_NOT_FOUND@ 0000000180004ce0     libclrfmodw001.obj
 0002:00000cf8       ??_C@_0BM@NHMCKHOB@JVMTI_ERROR_INVALID_MONITOR@ 0000000180004cf8     libclrfmodw001.obj
 0002:00000d18       ??_C@_0BO@PPEDAJGL@JVMTI_ERROR_NOT_MONITOR_OWNER@ 0000000180004d18     libclrfmodw001.obj
 0002:00000d38       ??_C@_0BG@FCAIPEID@JVMTI_ERROR_INTERRUPT@ 0000000180004d38     libclrfmodw001.obj
 0002:00000d50       ??_C@_0CB@EGDBNKOI@JVMTI_ERROR_INVALID_CLASS_FORMA@ 0000000180004d50     libclrfmodw001.obj
 0002:00000d78       ??_C@_0CG@DGKOGIAL@JVMTI_ERROR_CIRCULAR_CLASS_DEFI@ 0000000180004d78     libclrfmodw001.obj
 0002:00000da0       ??_C@_0BP@ICEALPKC@JVMTI_ERROR_FAILS_VERIFICATION@ 0000000180004da0     libclrfmodw001.obj
 0002:00000dc0       ??_C@_0DC@JDACLMIO@JVMTI_ERROR_UNSUPPORTED_REDEFIN@ 0000000180004dc0     libclrfmodw001.obj
 0002:00000df8       ??_C@_0DE@GKDKNOMJ@JVMTI_ERROR_UNSUPPORTED_REDEFIN@ 0000000180004df8     libclrfmodw001.obj
 0002:00000e30       ??_C@_0BO@LAFKIOG@JVMTI_ERROR_INVALID_TYPESTATE@ 0000000180004e30     libclrfmodw001.obj
 0002:00000e50       ??_C@_0DH@INDGCLLB@JVMTI_ERROR_UNSUPPORTED_REDEFIN@ 0000000180004e50     libclrfmodw001.obj
 0002:00000e88       ??_C@_0DE@NHEOMMGI@JVMTI_ERROR_UNSUPPORTED_REDEFIN@ 0000000180004e88     libclrfmodw001.obj
 0002:00000ec0       ??_C@_0CA@EKPNJOEP@JVMTI_ERROR_UNSUPPORTED_VERSION@ 0000000180004ec0     libclrfmodw001.obj
 0002:00000ee0       ??_C@_0BN@OFFMAHHL@JVMTI_ERROR_NAMES_DONT_MATCH@ 0000000180004ee0     libclrfmodw001.obj
 0002:00000f00       ??_C@_0DN@HHBBLAKE@JVMTI_ERROR_UNSUPPORTED_REDEFIN@ 0000000180004f00     libclrfmodw001.obj
 0002:00000f40       ??_C@_0DO@HMBGBGNA@JVMTI_ERROR_UNSUPPORTED_REDEFIN@ 0000000180004f40     libclrfmodw001.obj
 0002:00000f80       ??_C@_0BP@PBECGKHJ@JVMTI_ERROR_UNMODIFIABLE_CLASS@ 0000000180004f80     libclrfmodw001.obj
 0002:00000fa0       ??_C@_0BK@CANILEHF@JVMTI_ERROR_NOT_AVAILABLE@ 0000000180004fa0     libclrfmodw001.obj
 0002:00000fc0       ??_C@_0CE@INJKMEFK@JVMTI_ERROR_MUST_POSSESS_CAPABI@ 0000000180004fc0     libclrfmodw001.obj
 0002:00000fe8       ??_C@_0BJ@LBFPFPDM@JVMTI_ERROR_NULL_POINTER@ 0000000180004fe8     libclrfmodw001.obj
 0002:00001008       ??_C@_0BP@CHJPNNEM@JVMTI_ERROR_ABSENT_INFORMATION@ 0000000180005008     libclrfmodw001.obj
 0002:00001028       ??_C@_0BP@OMFMNLC@JVMTI_ERROR_INVALID_EVENT_TYPE@ 0000000180005028     libclrfmodw001.obj
 0002:00001048       ??_C@_0BN@BIBNPHHO@JVMTI_ERROR_ILLEGAL_ARGUMENT@ 0000000180005048     libclrfmodw001.obj
 0002:00001068       ??_C@_0BK@KKNDHDCE@JVMTI_ERROR_NATIVE_METHOD@ 0000000180005068     libclrfmodw001.obj
 0002:00001088       ??_C@_0BK@PMKCFHAE@JVMTI_ERROR_OUT_OF_MEMORY@ 0000000180005088     libclrfmodw001.obj
 0002:000010a8       ??_C@_0BK@NNJBDMNB@JVMTI_ERROR_ACCESS_DENIED@ 00000001800050a8     libclrfmodw001.obj
 0002:000010c8       ??_C@_0BI@GHECLMNC@JVMTI_ERROR_WRONG_PHASE@ 00000001800050c8     libclrfmodw001.obj
 0002:000010e0       ??_C@_0BF@OLIHJOII@JVMTI_ERROR_INTERNAL@ 00000001800050e0     libclrfmodw001.obj
 0002:000010f8       ??_C@_0BO@EOHGKJHI@JVMTI_ERROR_UNATTACHED_THREAD@ 00000001800050f8     libclrfmodw001.obj
 0002:00001118       ??_C@_0CA@LKHFDACL@JVMTI_ERROR_INVALID_ENVIRONMENT@ 0000000180005118     libclrfmodw001.obj
 0002:00001138       ??_C@_0BA@MMFHLOKK@?$DMunknown?5error?$DO@ 0000000180005138     libclrfmodw001.obj
 0002:00001148       ??_C@_0CF@CBHOKDB@throwable?5?$DN?5jni?9?$DOExceptionOccur@ 0000000180005148     libclrfmodw001.obj
 0002:00001170       ??_C@_03OFAPEBGM@?$CFs?6@  0000000180005170     libclrfmodw001.obj
 0002:00001178       ??_C@_0DM@LPIGEGNJ@s?2test?2hotspot?2jtreg?2vmTestbase@ 0000000180005178     libclrfmodw001.obj
 0002:000011b8       ??_C@_0CC@NFCNPEPK@Exception?5in?5JNI?5call?5?$CIcleared?$CJ@ 00000001800051b8     libclrfmodw001.obj
 0002:000011e0       ??_C@_0BJ@IBAKFIKF@jni?9?$DOExceptionDescribe?$CI?$CJ@ 00000001800051e0     libclrfmodw001.obj
 0002:00001200       ??_C@_0BG@GGKALKMH@jni?9?$DOExceptionClear?$CI?$CJ@ 0000000180005200     libclrfmodw001.obj
 0002:00001218       ??_C@_0CF@JMGFGJLJ@?$CD?5?5?5verified?5JNI?5assertion?5is?5F@ 0000000180005218     libclrfmodw001.obj
 0002:00001240       ??_C@_0CB@MLNJNCLJ@?5?5jvmti?5error?3?5code?$DN?$CFd?0?5name?$DN?$CFs@ 0000000180005240     libclrfmodw001.obj
 0002:00001268       ??_C@_0CD@OHBGDKMK@?$CD?5?5?5jvmti?5error?3?5code?$DN?$CFd?0?5name?$DN@ 0000000180005268     libclrfmodw001.obj
 0002:00001290       ??_C@_0CG@JNNCGPHB@?$CD?5?5?5error?5expected?3?5code?$DN?$CFd?0?5na@ 0000000180005290     libclrfmodw001.obj
 0002:000012c0       ??_C@_0EB@IMGKPCGE@?$CIstr_obj?5?$DN?5jni?9?$DONewStringUTF?$CIco@ 00000001800052c0     libclrfmodw001.obj
 0002:00001310       ??_C@_0EA@HFOGGBCC@s?2test?2hotspot?2jtreg?2vmTestbase@ 0000000180005310     libclrfmodw001.obj
 0002:00001350       ??_C@_05KKCIMGE@error@     0000000180005350     libclrfmodw001.obj
 0002:00001358       ??_C@_0CJ@JACLEAA@Test?5failed?5by?5setFailStatus?$CI?$CJ?4@ 0000000180005358     libclrfmodw001.obj
 0002:00001390       ??_C@_0EA@PNBCDMOA@s?2test?2hotspot?2jtreg?2vmTestbase@ 0000000180005390     libclrfmodw001.obj
 0002:000013d0       ??_C@_0DI@ILAHDLMP@?$CI?$CKagentThreadProc?$CJ?$CIjvmti_env?0?5a@ 00000001800053d0     libclrfmodw001.obj
 0002:00001408       ??_C@_0BD@KDBALNLB@JVMTI?5agent?5thread@ 0000000180005408     libclrfmodw001.obj
 0002:00001420       ??_C@_0BB@NOKBFPFO@java?1lang?1Thread@ 0000000180005420     libclrfmodw001.obj
 0002:00001434       ??_C@_06FALKBLGB@?$DMinit?$DO@ 0000000180005434     libclrfmodw001.obj
 0002:00001440       ??_C@_0BG@IKDDPPGD@?$CILjava?1lang?1String?$DL?$CJV@ 0000000180005440     libclrfmodw001.obj
 0002:00001460       ??_C@_0EB@IFJBFEKC@?$CIthreadClass?5?$DN?5jni_env?9?$DOFindCla@ 0000000180005460     libclrfmodw001.obj
 0002:000014b0       ??_C@_0GF@FGFIBKKL@?$CIthreadCtor?5?$DN?5jni_env?9?$DOGetMetho@ 00000001800054b0     libclrfmodw001.obj
 0002:00001518       ??_C@_0DN@NCPDJLOG@?$CIthreadName?5?$DN?5jni_env?9?$DONewStrin@ 0000000180005518     libclrfmodw001.obj
 0002:00001560       ??_C@_0FE@PFKODBGC@?$CIthreadObject?5?$DN?5jni_env?9?$DONewObj@ 0000000180005560     libclrfmodw001.obj
 0002:000015c0       ??_C@_0ED@HOBAHHJI@?$CIthreadGlobalRef?5?$DN?5jni_env?9?$DONew@ 00000001800055c0     libclrfmodw001.obj
 0002:00001610       ??_C@_0FN@HNJJAHFC@jvmti_env?9?$DORunAgentThread?$CIagent@ 0000000180005610     libclrfmodw001.obj
 0002:00001670       ??_C@_0EA@MOJDNKDF@Debuggee?5status?5sync?5aborted?5be@ 0000000180005670     libclrfmodw001.obj
 0002:000016b0       ??_C@_0EA@EEOEJAEN@status?5?$DN?5syncDebuggeeStatus?$CIjni@ 00000001800056b0     libclrfmodw001.obj
 0002:000016f0       ??_C@_0BL@JBCFNBMB@nsk_jvmti_resetAgentData?$CI?$CJ@ 00000001800056f0     libclrfmodw001.obj
 0002:00001710       ??_C@_0EL@LPBEELIP@s?2test?2hotspot?2jtreg?2vmTestbase@ 0000000180005710     libclrfmodw001.obj
 0002:00001760       ??_C@_0CK@JDAMFDMJ@jvmti?9?$DOSetTag?$CIo?0?5tag?$CJ?5?$DN?$DN?5JVMTI_@ 0000000180005760     libclrfmodw001.obj
 0002:00001790       ??_C@_0CC@DAMNHKNI@Can?8t?5set?5tag?5?$CFli?5for?5object?5?$CFl@ 0000000180005790     libclrfmodw001.obj
 0002:000017b8       ??_C@_0DL@HAJPNKEF@jvmti?9?$DOGetObjectHashCode?$CIo?0?5?$CGha@ 00000001800057b8     libclrfmodw001.obj
 0002:000017f8       ??_C@_0BL@JFPIEOBF@Can?8t?5get?5hash?5object?5?$CFlx?6@ 00000001800057f8     libclrfmodw001.obj
 0002:00001818       ??_C@_0BG@DICPHBKN@setTag?3?5?$CF08x?5?$DM?9?5?$CF?53li@ 0000000180005818     libclrfmodw001.obj
 0002:00001830       ??_C@_0DH@FCEEBDMJ@?$CIs?5?$DN?5jni?9?$DOGetStringUTFChars?$CIsIn@ 0000000180005830     libclrfmodw001.obj
 0002:00001868       ??_C@_0BJ@OKKGHDCN@Can?8t?5get?5string?5at?5?$CF?$CDp?6@ 0000000180005868     libclrfmodw001.obj
 0002:00001888       ??_C@_0BP@EKFLGGFJ@Can?8t?5get?5string?5at?5?$CF?$CDp?3?5null?6@ 0000000180005888     libclrfmodw001.obj
 0002:000018a8       ??_C@_06ICODBHCL@?5?1?1?5?$CFs@ 00000001800058a8     libclrfmodw001.obj
 0002:000018b0       ??_C@_0DB@KGFPLEGO@?$CIr?5?$DN?5jvmti?9?$DOGetTag?$CIo?0?5?$CGtag?$CJ?$CJ?5?$DN?$DN@ 00000001800058b0     libclrfmodw001.obj
 0002:000018e8       ??_C@_0CO@PDAGBCGJ@Can?8t?5GetTag?5for?5object?5?$CFlx?4?5Re@ 00000001800058e8     libclrfmodw001.obj
 0002:00001918       ??_C@_0CH@HPEODOHC@TEST_BUG?3?5Max?4?5number?5of?5refs?5r@ 0000000180005918     libclrfmodw001.obj
 0002:00001940       ??_C@_0DI@PHFCABIM@?$CIr?5?$DN?5jvmti?9?$DOGetTag?$CIfrom?0?5?$CGtagFr@ 0000000180005940     libclrfmodw001.obj
 0002:00001978       ??_C@_0DI@MDEGFNKD@TEST_BUG?3?5Can?8t?5GetTag?5for?5obje@ 0000000180005978     libclrfmodw001.obj
 0002:000019b0       ??_C@_0DE@MLELJAHM@?$CIr?5?$DN?5jvmti?9?$DOGetTag?$CIto?0?5?$CGtagTo?$CJ?$CJ@ 00000001800059b0     libclrfmodw001.obj
 0002:000019e4       ??_C@_03CEMDFJG@Set@       00000001800059e4     libclrfmodw001.obj
 0002:000019e8       ??_C@_05MDNHABIA@Clear@    00000001800059e8     libclrfmodw001.obj
 0002:000019f0       ??_C@_0DJ@KPGCFJJP@?$CI?$CFsFieldModificationWatch?$CD?$CFd?$CJ?5u@ 00000001800059f0     libclrfmodw001.obj
 0002:00001a30       ??_C@_0CK@DEFLIKCM@Wrong?5result?5of?5a?5valid?5call?5to@ 0000000180005a30     libclrfmodw001.obj
 0002:00001a60       ??_C@_0DG@LAJPGIIE@?$CIGetPotentialCapabilities?$CJ?5unex@ 0000000180005a60     libclrfmodw001.obj
 0002:00001a98       ??_C@_0CN@LKPEOJPO@?$CIAddCapabilities?$CJ?5unexpected?5er@ 0000000180005a98     libclrfmodw001.obj
 0002:00001ac8       ??_C@_0CN@BCCBOHCH@?$CIGetCapabilities?$CJ?5unexpected?5er@ 0000000180005ac8     libclrfmodw001.obj
 0002:00001af8       ??_C@_0CP@IMINGNLL@?$CISetEventCallbacks?$CJ?5unexpected?5@ 0000000180005af8     libclrfmodw001.obj
 0002:00001b28       ??_C@_0DK@JGGEPECM@Failed?5to?5enable?5JVMTI_EVENT_FI@ 0000000180005b28     libclrfmodw001.obj
 0002:00001b68       ??_C@_0DF@JEIOMCOG@Warning?3?5FieldModification?5watc@ 0000000180005b68     libclrfmodw001.obj
 0002:00001ba0       ??_C@_0M@HPIAONLC@?$CIField?5?$CFd?$CJ?5@ 0000000180005ba0     libclrfmodw001.obj
 0002:00001bb0       ??_C@_0DI@CNGPLGLM@FieldModification?5event?5without@ 0000000180005bb0     libclrfmodw001.obj
 0002:00001be8       ??_C@_0DG@NAFMPMGP@?$CIField?5?$CFd?$CJ?5thrown?5field?5ID?5expe@ 0000000180005be8     libclrfmodw001.obj
 0002:00001c30       ??_C@_1EC@JIJBPKFM@?$AAa?$AAp?$AAi?$AA?9?$AAm?$AAs?$AA?9?$AAw?$AAi?$AAn?$AA?9?$AAc?$AAo?$AAr?$AAe@ 0000000180005c30     MSVCRT:thread_safe_statics.obj
 0002:00001c78       ??_C@_1BK@MGMFAEKH@?$AAk?$AAe?$AAr?$AAn?$AAe?$AAl?$AA3?$AA2?$AA?4?$AAd?$AAl?$AAl@ 0000000180005c78     MSVCRT:thread_safe_statics.obj
 0002:00001c98       ??_C@_0BJ@JEBJOJFJ@SleepConditionVariableCS@ 0000000180005c98     MSVCRT:thread_safe_statics.obj
 0002:00001cb8       ??_C@_0BJ@PGPPEPCC@WakeAllConditionVariable@ 0000000180005cb8     MSVCRT:thread_safe_statics.obj
 0002:00001cd8       _pDefaultRawDllMain        0000000180005cd8     MSVCRT:dll_dllmain.obj
 0002:00001cd8       _pRawDllMain               0000000180005cd8     MSVCRT:dll_dllmain.obj
 0002:00001ce0       __xmm@ffffffffffffffffffffffffffffffff 0000000180005ce0     MSVCRT:utility.obj
 0002:00001cf0       _load_config_used          0000000180005cf0     MSVCRT:loadcfg.obj
 0002:00001f00       _tls_used                  0000000180005f00     MSVCRT:tlssup.obj
 0002:00001f28       __volatile_metadata        0000000180005f28     <linker-defined>
 0002:000022e8       __rtc_iaa                  00000001800062e8     MSVCRT:initsect.obj
 0002:000022f0       __rtc_izz                  00000001800062f0     MSVCRT:initsect.obj
 0002:000022f8       __rtc_taa                  00000001800062f8     MSVCRT:initsect.obj
 0002:00002300       __rtc_tzz                  0000000180006300     MSVCRT:initsect.obj
 0002:00002308       _tls_start                 0000000180006308     MSVCRT:tlssup.obj
 0002:0000230c       _Init_thread_epoch         000000018000630c     MSVCRT:thread_safe_statics.obj
 0002:00002310       _tls_end                   0000000180006310     MSVCRT:tlssup.obj
 0002:00002ad4       __IMPORT_DESCRIPTOR_KERNEL32 0000000180006ad4     kernel32:KERNEL32.dll
 0002:00002ae8       __IMPORT_DESCRIPTOR_VCRUNTIME140 0000000180006ae8     vcruntime:VCRUNTIME140.dll
 0002:00002afc       __IMPORT_DESCRIPTOR_api-ms-win-crt-runtime-l1-1-0 0000000180006afc     ucrt:api-ms-win-crt-runtime-l1-1-0.dll
 0002:00002b10       __IMPORT_DESCRIPTOR_api-ms-win-crt-stdio-l1-1-0 0000000180006b10     ucrt:api-ms-win-crt-stdio-l1-1-0.dll
 0002:00002b24       __IMPORT_DESCRIPTOR_api-ms-win-crt-string-l1-1-0 0000000180006b24     ucrt:api-ms-win-crt-string-l1-1-0.dll
 0002:00002b38       __NULL_IMPORT_DESCRIPTOR   0000000180006b38     kernel32:KERNEL32.dll
 0003:000000f8       _Init_global_epoch         00000001800080f8     MSVCRT:thread_safe_statics.obj
 0003:00000100       __security_cookie          0000000180008100     MSVCRT:gs_cookie.obj
 0003:00000108       __security_cookie_complement 0000000180008108     MSVCRT:gs_cookie.obj
 0003:00000110       __scrt_native_dllmain_reason 0000000180008110     MSVCRT:utility.obj
 0003:00000118       __isa_available            0000000180008118     MSVCRT:cpu_disp.obj
 0003:0000011c       __isa_enabled              000000018000811c     MSVCRT:cpu_disp.obj
 0003:00000120       __memset_fast_string_threshold 0000000180008120     MSVCRT:cpu_disp.obj
 0003:00000128       __memset_nt_threshold      0000000180008128     MSVCRT:cpu_disp.obj
 0003:00000130       __scrt_ucrt_dll_is_in_use  0000000180008130     MSVCRT:ucrt_stubs.obj
 0003:00000140       g_wrongHeapCallbacks       0000000180008140     libclrfmodw001.obj
 0003:000001c0       g_szTagInfo                00000001800081c0     libclrfmodw001.obj
 0003:00002100       g_tagFlags                 000000018000a100     libclrfmodw001.obj
 0003:000024e8       g_refsToVerifyCnt          000000018000a4e8     libclrfmodw001.obj
 0003:000024ec       g_fakeUserData             000000018000a4ec     libclrfmodw001.obj
 0003:000024f0       g_tagVisitCount            000000018000a4f0     libclrfmodw001.obj
 0003:00003490       g_refsToVerify             000000018000b490     libclrfmodw001.obj
 0003:0001ab90       g_userDataError            0000000180022b90     libclrfmodw001.obj
 0003:0001ae80       ?_OptionsStorage@?1??__local_stdio_printf_options@@9@4_KA 0000000180022e80     libclrfmodw001.obj
 0003:0001b448       _tls_index                 0000000180023448     MSVCRT:tlssup.obj
 0003:0001b450       __scrt_current_native_startup_state 0000000180023450     MSVCRT:utility.obj
 0003:0001b458       __scrt_native_startup_lock 0000000180023458     MSVCRT:utility.obj
 0003:0001b498       __scrt_debugger_hook_flag  0000000180023498     MSVCRT:utility_desktop.obj
 0003:0001b4a0       ?__type_info_root_node@@3U__type_info_node@@A 00000001800234a0     MSVCRT:tncleanup.obj
 0003:0001b4b0       ?_OptionsStorage@?1??__local_stdio_scanf_options@@9@4_KA 00000001800234b0     MSVCRT:default_local_stdio_options.obj
 0003:0001b4b8       __favor                    00000001800234b8     MSVCRT:cpu_disp.obj
 0003:0001b4c0       __dyn_tls_init_callback    00000001800234c0     <common>

 entry point at        0001:000023e0

 Static symbols

 0000:fffda000       .debug$S                   0000000180000000     clrfmodw001.exp
 0000:fffda000       .debug$S                   0000000180000000     vcruntime:VCRUNTIME140.dll
 0000:fffda000       .debug$S                   0000000180000000     vcruntime:VCRUNTIME140.dll
 0000:fffda000       .debug$S                   0000000180000000     vcruntime:VCRUNTIME140.dll
 0000:fffda000       .debug$S                   0000000180000000     vcruntime:VCRUNTIME140.dll
 0000:fffda000       .debug$S                   0000000180000000     vcruntime:VCRUNTIME140.dll
 0000:fffda000       .debug$S                   0000000180000000     vcruntime:VCRUNTIME140.dll
 0000:fffda000       .debug$S                   0000000180000000     vcruntime:VCRUNTIME140.dll
 0000:fffda000       .debug$S                   0000000180000000     ucrt:api-ms-win-crt-convert-l1-1-0.dll
 0002:ffffc000       .idata$6                   0000000180000000     ucrt:api-ms-win-crt-convert-l1-1-0.dll
 0000:fffda000       .debug$S                   0000000180000000     ucrt:api-ms-win-crt-heap-l1-1-0.dll
 0000:fffda000       .debug$S                   0000000180000000     ucrt:api-ms-win-crt-heap-l1-1-0.dll
 0000:fffda000       .debug$S                   0000000180000000     ucrt:api-ms-win-crt-heap-l1-1-0.dll
 0000:fffda000       .debug$S                   0000000180000000     ucrt:api-ms-win-crt-heap-l1-1-0.dll
 0002:ffffc000       .idata$6                   0000000180000000     ucrt:api-ms-win-crt-heap-l1-1-0.dll
 0000:fffda000       .debug$S                   0000000180000000     ucrt:api-ms-win-crt-runtime-l1-1-0.dll
 0000:fffda000       .debug$S                   0000000180000000     ucrt:api-ms-win-crt-runtime-l1-1-0.dll
 0000:fffda000       .debug$S                   0000000180000000     ucrt:api-ms-win-crt-runtime-l1-1-0.dll
 0000:fffda000       .debug$S                   0000000180000000     ucrt:api-ms-win-crt-runtime-l1-1-0.dll
 0000:fffda000       .debug$S                   0000000180000000     ucrt:api-ms-win-crt-runtime-l1-1-0.dll
 0000:fffda000       .debug$S                   0000000180000000     ucrt:api-ms-win-crt-runtime-l1-1-0.dll
 0000:fffda000       .debug$S                   0000000180000000     ucrt:api-ms-win-crt-runtime-l1-1-0.dll
 0000:fffda000       .debug$S                   0000000180000000     ucrt:api-ms-win-crt-runtime-l1-1-0.dll
 0000:fffda000       .debug$S                   0000000180000000     ucrt:api-ms-win-crt-runtime-l1-1-0.dll
 0000:fffda000       .debug$S                   0000000180000000     ucrt:api-ms-win-crt-runtime-l1-1-0.dll
 0000:fffda000       .debug$S                   0000000180000000     ucrt:api-ms-win-crt-runtime-l1-1-0.dll
 0000:fffda000       .debug$S                   0000000180000000     ucrt:api-ms-win-crt-runtime-l1-1-0.dll
 0000:fffda000       .debug$S                   0000000180000000     ucrt:api-ms-win-crt-runtime-l1-1-0.dll
 0000:fffda000       .debug$S                   0000000180000000     ucrt:api-ms-win-crt-runtime-l1-1-0.dll
 0000:fffda000       .debug$S                   0000000180000000     ucrt:api-ms-win-crt-runtime-l1-1-0.dll
 0000:fffda000       .debug$S                   0000000180000000     ucrt:api-ms-win-crt-runtime-l1-1-0.dll
 0000:fffda000       .debug$S                   0000000180000000     ucrt:api-ms-win-crt-stdio-l1-1-0.dll
 0000:fffda000       .debug$S                   0000000180000000     ucrt:api-ms-win-crt-stdio-l1-1-0.dll
 0000:fffda000       .debug$S                   0000000180000000     ucrt:api-ms-win-crt-stdio-l1-1-0.dll
 0000:fffda000       .debug$S                   0000000180000000     ucrt:api-ms-win-crt-stdio-l1-1-0.dll
 0000:fffda000       .debug$S                   0000000180000000     ucrt:api-ms-win-crt-stdio-l1-1-0.dll
 0000:fffda000       .debug$S                   0000000180000000     ucrt:api-ms-win-crt-stdio-l1-1-0.dll
 0000:fffda000       .debug$S                   0000000180000000     ucrt:api-ms-win-crt-stdio-l1-1-0.dll
 0000:fffda000       .debug$S                   0000000180000000     ucrt:api-ms-win-crt-stdio-l1-1-0.dll
 0000:fffda000       .debug$S                   0000000180000000     ucrt:api-ms-win-crt-stdio-l1-1-0.dll
 0000:fffda000       .debug$S                   0000000180000000     ucrt:api-ms-win-crt-stdio-l1-1-0.dll
 0000:fffda000       .debug$S                   0000000180000000     ucrt:api-ms-win-crt-string-l1-1-0.dll
 0000:fffda000       .debug$S                   0000000180000000     ucrt:api-ms-win-crt-string-l1-1-0.dll
 0000:fffda000       .debug$S                   0000000180000000     ucrt:api-ms-win-crt-string-l1-1-0.dll
 0000:fffda000       .debug$S                   0000000180000000     ucrt:api-ms-win-crt-string-l1-1-0.dll
 0000:fffda000       .debug$S                   0000000180000000     ucrt:api-ms-win-crt-string-l1-1-0.dll
 0000:fffda000       .debug$S                   0000000180000000     ucrt:api-ms-win-crt-string-l1-1-0.dll
 0000:fffda000       .debug$S                   0000000180000000     ucrt:api-ms-win-crt-string-l1-1-0.dll
 0000:fffda000       .debug$S                   0000000180000000     ucrt:api-ms-win-crt-string-l1-1-0.dll
 0000:fffda000       .debug$S                   0000000180000000     kernel32:KERNEL32.dll
 0000:fffda000       .debug$S                   0000000180000000     kernel32:KERNEL32.dll
 0000:fffda000       .debug$S                   0000000180000000     kernel32:KERNEL32.dll
 0000:fffda000       .debug$S                   0000000180000000     kernel32:KERNEL32.dll
 0000:fffda000       .debug$S                   0000000180000000     kernel32:KERNEL32.dll
 0000:fffda000       .debug$S                   0000000180000000     kernel32:KERNEL32.dll
 0000:fffda000       .debug$S                   0000000180000000     kernel32:KERNEL32.dll
 0000:fffda000       .debug$S                   0000000180000000     kernel32:KERNEL32.dll
 0000:fffda000       .debug$S                   0000000180000000     kernel32:KERNEL32.dll
 0000:fffda000       .debug$S                   0000000180000000     kernel32:KERNEL32.dll
 0000:fffda000       .debug$S                   0000000180000000     kernel32:KERNEL32.dll
 0000:fffda000       .debug$S                   0000000180000000     kernel32:KERNEL32.dll
 0000:fffda000       .debug$S                   0000000180000000     kernel32:KERNEL32.dll
 0000:fffda000       .debug$S                   0000000180000000     kernel32:KERNEL32.dll
 0000:fffda000       .debug$S                   0000000180000000     kernel32:KERNEL32.dll
 0000:fffda000       .debug$S                   0000000180000000     kernel32:KERNEL32.dll
 0000:fffda000       .debug$S                   0000000180000000     kernel32:KERNEL32.dll
 0000:fffda000       .debug$S                   0000000180000000     kernel32:KERNEL32.dll
 0000:fffda000       .debug$S                   0000000180000000     kernel32:KERNEL32.dll
 0000:fffda000       .debug$S                   0000000180000000     kernel32:KERNEL32.dll
 0000:fffda000       .debug$S                   0000000180000000     kernel32:KERNEL32.dll
 0000:fffda000       .debug$S                   0000000180000000     kernel32:KERNEL32.dll
 0000:fffda000       .debug$S                   0000000180000000     kernel32:KERNEL32.dll
 0000:fffda000       .debug$S                   0000000180000000     kernel32:KERNEL32.dll
 0000:fffda000       .debug$S                   0000000180000000     kernel32:KERNEL32.dll
 0000:fffda000       .debug$S                   0000000180000000     kernel32:KERNEL32.dll
 0000:fffda000       .debug$S                   0000000180000000     kernel32:KERNEL32.dll
 0000:fffda000       .debug$S                   0000000180000000     kernel32:KERNEL32.dll
 0001:00000ec8       addRefToVerify             0000000180001ec8 f   libclrfmodw001.obj
 0001:00000f34       agentThreadWrapper         0000000180001f34 f   libclrfmodw001.obj
 0001:00001124       file_basename              0000000180002124 f   libclrfmodw001.obj
 0001:00001790       startAgentThreadWrapper    0000000180002790 f   libclrfmodw001.obj
 0001:00001bfc       syncDebuggeeStatus         0000000180002bfc f   libclrfmodw001.obj
 0001:00001e9c       capture_previous_context   0000000180002e9c f   MSVCRT:gs_report.obj
 0001:00001f10       ?__scrt_initialize_thread_safe_statics@@YAHXZ 0000000180002f10 f   MSVCRT:thread_safe_statics.obj
 0001:00001fe0       ?__scrt_uninitialize_thread_safe_statics@@YAXXZ 0000000180002fe0 f   MSVCRT:thread_safe_statics.obj
 0001:00002090       $$000000                   0000000180003090     MSVCRT:amdsecgs.obj
 0001:000020c0       ?dllmain_crt_dispatch@@YAHQEAUHINSTANCE__@@KQEAX@Z 00000001800030c0 f   MSVCRT:dll_dllmain.obj
 0001:00002110       ?dllmain_crt_process_attach@@YAHQEAUHINSTANCE__@@QEAX@Z 0000000180003110 f   MSVCRT:dll_dllmain.obj
 0001:00002228       ?dllmain_crt_process_detach@@YAH_N@Z 0000000180003228 f   MSVCRT:dll_dllmain.obj
 0001:000022ac       ?dllmain_dispatch@@YAHQEAUHINSTANCE__@@KQEAX@Z 00000001800032ac f   MSVCRT:dll_dllmain.obj
 0001:00002cc0       $$000000                   0000000180003cc0     MSVCRT:guard_dispatch.obj
 0001:00002ce0       $$000000                   0000000180003ce0     MSVCRT:guard_xfg_dispatch.obj
 0001:00002cf6       ?fin$0@?0??dllmain_crt_process_attach@@YAHQEAUHINSTANCE__@@QEAX@Z@4HA 0000000180003cf6 f   MSVCRT:dll_dllmain.obj
 0001:00002d0d       ?fin$0@?0??dllmain_crt_process_detach@@YAH_N@Z@4HA 0000000180003d0d f   MSVCRT:dll_dllmain.obj
 0001:00002d26       ?fin$1@?0??dllmain_crt_process_detach@@YAH_N@Z@4HA 0000000180003d26 f   MSVCRT:dll_dllmain.obj
 0001:00002d3a       ?filt$0@?0??dllmain_dispatch@@YAHQEAUHINSTANCE__@@KQEAX@Z@4HA 0000000180003d3a f   MSVCRT:dll_dllmain.obj
 0001:00002d70       __scrt_is_nonwritable_in_current_image$filt$0 0000000180003d70 f   MSVCRT:utility.obj
 0002:000001e0       ?__scrt_initialize_tss_var@@3P6AHXZEA 00000001800041e0     MSVCRT:thread_safe_statics.obj
 0002:00000300       ?opcLengths@@3QBEB         0000000180004300     libclrfmodw001.obj
 0002:00001c20       GS_ExceptionPointers       0000000180005c20     MSVCRT:gs_report.obj
 0002:00002318       $unwind$fprintf            0000000180006318     libclrfmodw001.obj
 0002:00002324       $unwind$printf             0000000180006324     libclrfmodw001.obj
 0002:00002330       $unwind$?NewObject@JNIEnv_@@QEAAPEAV_jobject@@PEAV_jclass@@PEAU_jmethodID@@ZZ 0000000180006330     libclrfmodw001.obj
 0002:00002330       $unwind$nsk_lcomplain      0000000180006330     libclrfmodw001.obj
 0002:00002330       $unwind$nsk_ldisplay       0000000180006330     libclrfmodw001.obj
 0002:00002338       $unwind$nsk_lvdisplay      0000000180006338     libclrfmodw001.obj
 0002:00002338       $unwind$_RTC_Initialize    0000000180006338     MSVCRT:initsect.obj
 0002:00002338       $unwind$_RTC_Terminate     0000000180006338     MSVCRT:initsect.obj
 0002:00002338       $unwind$?__scrt_initialize_thread_safe_statics@@YAHXZ 0000000180006338     MSVCRT:thread_safe_statics.obj
 0002:00002344       $unwind$nsk_lvcomplain     0000000180006344     libclrfmodw001.obj
 0002:0000235c       $unwind$nsk_ltrace         000000018000635c     libclrfmodw001.obj
 0002:0000235c       $unwind$__report_gsfailure 000000018000635c     MSVCRT:gs_report.obj
 0002:00002364       $unwind$Agent_Initialize   0000000180006364     libclrfmodw001.obj
 0002:00002364       $unwind$nsk_lvtrace        0000000180006364     libclrfmodw001.obj
 0002:00002364       $unwind$__raise_securityfailure 0000000180006364     MSVCRT:gs_report.obj
 0002:00002364       $unwind$__scrt_initialize_crt 0000000180006364     MSVCRT:utility.obj
 0002:00002364       $unwind$__scrt_initialize_onexit_tables 0000000180006364     MSVCRT:utility.obj
 0002:00002364       $unwind$__scrt_release_startup_lock 0000000180006364     MSVCRT:utility.obj
 0002:00002364       $unwind$__scrt_uninitialize_crt 0000000180006364     MSVCRT:utility.obj
 0002:00002364       $unwind$_onexit            0000000180006364     MSVCRT:utility.obj
 0002:0000236c       $unwind$nsk_lverify        000000018000636c     libclrfmodw001.obj
 0002:0000237c       $unwind$nsk_vprintf        000000018000637c     libclrfmodw001.obj
 0002:0000238c       $unwind$nsk_printf         000000018000638c     libclrfmodw001.obj
 0002:00002394       $unwind$?nsk_jni_lverify@@YAHHPEAUJNIEnv_@@HQEBDH1ZZ 0000000180006394     libclrfmodw001.obj
 0002:000023a8       $unwind$?nsk_jni_check_exception@@YAHPEAUJNIEnv_@@QEBDH@Z 00000001800063a8     libclrfmodw001.obj
 0002:000023c4       $unwind$Java_nsk_jvmti_ClearFieldModificationWatch_clrfmodw001_check 00000001800063c4     libclrfmodw001.obj
 0002:000023c4       $unwind$Java_nsk_jvmti_unit_FollowReferences_FollowRefObjects_resetTags 00000001800063c4     libclrfmodw001.obj
 0002:000023c4       $unwind$addRefToVerify     00000001800063c4     libclrfmodw001.obj
 0002:000023c4       $unwind$nsk_jvmti_resetAgentData 00000001800063c4     libclrfmodw001.obj
 0002:000023c4       $unwind$nsk_jvmti_setFailStatus 00000001800063c4     libclrfmodw001.obj
 0002:000023c4       $unwind$__scrt_initialize_default_local_stdio_options 00000001800063c4     MSVCRT:default_local_stdio_options.obj
 0002:000023c4       $unwind$?dllmain_crt_dispatch@@YAHQEAUHINSTANCE__@@KQEAX@Z 00000001800063c4     MSVCRT:dll_dllmain.obj
 0002:000023c4       $unwind$DllMain            00000001800063c4     MSVCRT:dll_dllmain_stub.obj
 0002:000023c4       $unwind$__GSHandlerCheck   00000001800063c4     MSVCRT:gshandler.obj
 0002:000023c4       $unwind$?__scrt_uninitialize_thread_safe_statics@@YAXXZ 00000001800063c4     MSVCRT:thread_safe_statics.obj
 0002:000023c4       $unwind$__scrt_acquire_startup_lock 00000001800063c4     MSVCRT:utility.obj
 0002:000023c4       $unwind$__scrt_dllmain_after_initialize_c 00000001800063c4     MSVCRT:utility.obj
 0002:000023c4       $unwind$__scrt_dllmain_before_initialize_c 00000001800063c4     MSVCRT:utility.obj
 0002:000023c4       $unwind$__scrt_dllmain_crt_thread_attach 00000001800063c4     MSVCRT:utility.obj
 0002:000023c4       $unwind$__scrt_dllmain_crt_thread_detach 00000001800063c4     MSVCRT:utility.obj
 0002:000023c4       $unwind$__scrt_dllmain_uninitialize_c 00000001800063c4     MSVCRT:utility.obj
 0002:000023c4       $unwind$__scrt_dllmain_uninitialize_critical 00000001800063c4     MSVCRT:utility.obj
 0002:000023c4       $unwind$atexit             00000001800063c4     MSVCRT:utility.obj
 0002:000023cc       $unwind$nsk_jvmti_lverify  00000001800063cc     libclrfmodw001.obj
 0002:000023e0       $unwind$exitOnError        00000001800063e0     libclrfmodw001.obj
 0002:000023f0       $unwind$Java_nsk_share_jvmti_ArgumentHandler_getAgentOptionsString 00000001800063f0     libclrfmodw001.obj
 0002:00002404       $unwind$Java_nsk_jvmti_unit_FollowReferences_FollowRefObjects_getTag 0000000180006404     libclrfmodw001.obj
 0002:00002404       $unwind$Java_nsk_share_jvmti_DebugeeClass_checkStatus 0000000180006404     libclrfmodw001.obj
 0002:00002404       $unwind$agentThreadWrapper 0000000180006404     libclrfmodw001.obj
 0002:00002414       $unwind$startAgentThreadWrapper 0000000180006414     libclrfmodw001.obj
 0002:00002430       $unwind$syncDebuggeeStatus 0000000180006430     libclrfmodw001.obj
 0002:00002430       $unwind$__scrt_dllmain_exception_filter 0000000180006430     MSVCRT:utility.obj
 0002:00002444       $unwind$Java_nsk_share_jvmti_DebugeeClass_resetAgentData 0000000180006444     libclrfmodw001.obj
 0002:0000244c       $unwind$MA_checkStatus     000000018000644c     libclrfmodw001.obj
 0002:00002460       $unwind$Java_nsk_jvmti_unit_FollowReferences_FollowRefObjects_setTag 0000000180006460     libclrfmodw001.obj
 0002:00002478       $unwind$Java_nsk_jvmti_unit_FollowReferences_FollowRefObjects_addRefToVerify 0000000180006478     libclrfmodw001.obj
 0002:00002494       $unwind$switchWatch        0000000180006494     libclrfmodw001.obj
 0002:000024ac       $unwind$capture_previous_context 00000001800064ac     MSVCRT:gs_report.obj
 0002:000024b8       $unwind$__GSHandlerCheckCommon 00000001800064b8     MSVCRT:gshandler.obj
 0002:000024c0       $xdatasym                  00000001800064c0     MSVCRT:amdsecgs.obj
 0002:000024c4       $unwind$?dllmain_crt_process_attach@@YAHQEAUHINSTANCE__@@QEAX@Z 00000001800064c4     MSVCRT:dll_dllmain.obj
 0002:00002500       $unwind$?fin$0@?0??dllmain_crt_process_attach@@YAHQEAUHINSTANCE__@@QEAX@Z@4HA 0000000180006500     MSVCRT:dll_dllmain.obj
 0002:00002500       $unwind$?fin$0@?0??dllmain_crt_process_detach@@YAH_N@Z@4HA 0000000180006500     MSVCRT:dll_dllmain.obj
 0002:00002500       $unwind$?fin$1@?0??dllmain_crt_process_detach@@YAH_N@Z@4HA 0000000180006500     MSVCRT:dll_dllmain.obj
 0002:00002508       $unwind$?dllmain_crt_process_detach@@YAH_N@Z 0000000180006508     MSVCRT:dll_dllmain.obj
 0002:0000255c       $unwind$?dllmain_dispatch@@YAHQEAUHINSTANCE__@@KQEAX@Z 000000018000655c     MSVCRT:dll_dllmain.obj
 0002:00002584       $unwind$?filt$0@?0??dllmain_dispatch@@YAHQEAUHINSTANCE__@@KQEAX@Z@4HA 0000000180006584     MSVCRT:dll_dllmain.obj
 0002:0000258c       $unwind$_DllMainCRTStartup 000000018000658c     MSVCRT:dll_dllmain.obj
 0002:0000259c       $unwind$__scrt_is_nonwritable_in_current_image 000000018000659c     MSVCRT:utility.obj
 0002:000025bc       $unwind$__scrt_is_nonwritable_in_current_image$filt$0 00000001800065bc     MSVCRT:utility.obj
 0002:000025c4       $unwind$__scrt_fastfail    00000001800065c4     MSVCRT:utility_desktop.obj
 0002:000025d4       $unwind$__security_init_cookie 00000001800065d4     MSVCRT:gs_support.obj
 0002:000025e0       $unwind$__isa_available_init 00000001800065e0     MSVCRT:cpu_disp.obj
 0002:000025f0       $xdatasym                  00000001800065f0     MSVCRT:guard_dispatch.obj
 0002:000025f8       $xdatasym                  00000001800065f8     MSVCRT:guard_xfg_dispatch.obj
 0002:00002600       .edata                     0000000180006600     clrfmodw001.exp
 0002:00002628       rgpv                       0000000180006628     clrfmodw001.exp
 0002:00002674       rgszName                   0000000180006674     clrfmodw001.exp
 0002:000026c0       rgwOrd                     00000001800066c0     clrfmodw001.exp
 0002:000026e6       szName                     00000001800066e6     clrfmodw001.exp
 0002:000026f6       $N00001                    00000001800066f6     clrfmodw001.exp
 0002:00002705       $N00002                    0000000180006705     clrfmodw001.exp
 0002:00002712       $N00003                    0000000180006712     clrfmodw001.exp
 0002:0000274f       $N00004                    000000018000674f     clrfmodw001.exp
 0002:00002791       $N00005                    0000000180006791     clrfmodw001.exp
 0002:000027cf       $N00006                    00000001800067cf     clrfmodw001.exp
 0002:0000280f       $N00007                    000000018000680f     clrfmodw001.exp
 0002:00002850       $N00008                    0000000180006850     clrfmodw001.exp
 0002:00002895       $N00009                    0000000180006895     clrfmodw001.exp
 0002:000028d2       $N00010                    00000001800068d2     clrfmodw001.exp
 0002:0000291a       $N00011                    000000018000691a     clrfmodw001.exp
 0002:0000295a       $N00012                    000000018000695a     clrfmodw001.exp
 0002:00002997       $N00013                    0000000180006997     clrfmodw001.exp
 0002:000029d2       $N00014                    00000001800069d2     clrfmodw001.exp
 0002:00002a00       $N00015                    0000000180006a00     clrfmodw001.exp
 0002:00002a31       $N00016                    0000000180006a31     clrfmodw001.exp
 0002:00002a60       $N00017                    0000000180006a60     clrfmodw001.exp
 0002:00002a8f       $N00018                    0000000180006a8f     clrfmodw001.exp
 0002:00002ac4       $N00019                    0000000180006ac4     clrfmodw001.exp
 0002:00002eca       .idata$6                   0000000180006eca     kernel32:KERNEL32.dll
 0002:00002f2e       .idata$6                   0000000180006f2e     vcruntime:VCRUNTIME140.dll
 0002:00003090       .idata$6                   0000000180007090     ucrt:api-ms-win-crt-runtime-l1-1-0.dll
 0002:000030b2       .idata$6                   00000001800070b2     ucrt:api-ms-win-crt-stdio-l1-1-0.dll
 0002:000030d2       .idata$6                   00000001800070d2     ucrt:api-ms-win-crt-string-l1-1-0.dll
 0003:00000000       ?codeAttributeName@@3PEBDEB 0000000180008000     libclrfmodw001.obj
 0003:00000008       ?lineNumberAttributeName@@3PEBDEB 0000000180008008     libclrfmodw001.obj
 0003:00000010       ?localVarAttributeName@@3PEBDEB 0000000180008010     libclrfmodw001.obj
 0003:00000018       ?localVarTypeAttributeName@@3PEBDEB 0000000180008018     libclrfmodw001.obj
 0003:00000020       ?stackMapAttributeName@@3PEBDEB 0000000180008020     libclrfmodw001.obj
 0003:00000028       ?callBytes@@3PAEA          0000000180008028     libclrfmodw001.obj
 0003:0000002c       ?allocBytes@@3PAEA         000000018000802c     libclrfmodw001.obj
 0003:00000030       fields                     0000000180008030     libclrfmodw001.obj
 0003:0001ab94       redefineAttempted          0000000180022b94     libclrfmodw001.obj
 0003:0001ab98       nsk_context                0000000180022b98     libclrfmodw001.obj
 0003:0001aba4       redefineSucceed            0000000180022ba4     libclrfmodw001.obj
 0003:0001aba8       agentFailed                0000000180022ba8     libclrfmodw001.obj
 0003:0001abac       currentAgentStatus         0000000180022bac     libclrfmodw001.obj
 0003:0001abb0       context                    0000000180022bb0     libclrfmodw001.obj
 0003:0001ac68       agentThread                0000000180022c68     libclrfmodw001.obj
 0003:0001ac70       agentThreadProc            0000000180022c70     libclrfmodw001.obj
 0003:0001ac78       agentThreadArg             0000000180022c78     libclrfmodw001.obj
 0003:0001ac80       agent_data                 0000000180022c80     libclrfmodw001.obj
 0003:0001ac90       jvmti_env                  0000000180022c90     libclrfmodw001.obj
 0003:0001ac98       jvm                        0000000180022c98     libclrfmodw001.obj
 0003:0001aca0       jni_env                    0000000180022ca0     libclrfmodw001.obj
 0003:0001aca8       checkStatus_func           0000000180022ca8     libclrfmodw001.obj
 0003:0001acb0       ?codeAttributeIndex@@3GA   0000000180022cb0     libclrfmodw001.obj
 0003:0001acb4       ?lineNumberAttributeIndex@@3GA 0000000180022cb4     libclrfmodw001.obj
 0003:0001acb8       ?localVarAttributeIndex@@3GA 0000000180022cb8     libclrfmodw001.obj
 0003:0001acbc       ?localVarTypeAttributeIndex@@3GA 0000000180022cbc     libclrfmodw001.obj
 0003:0001acc0       ?stackMapAttributeIndex@@3GA 0000000180022cc0     libclrfmodw001.obj
 0003:0001acc4       ?stackFrameOffset@@3GA     0000000180022cc4     libclrfmodw001.obj
 0003:0001acc8       ?mode@@3HA                 0000000180022cc8     libclrfmodw001.obj
 0003:0001accc       ?constantPoolSize@@3GA     0000000180022ccc     libclrfmodw001.obj
 0003:0001acd0       ?orig@@3PEBEEB             0000000180022cd0     libclrfmodw001.obj
 0003:0001acd8       ?gen@@3PEAEEA              0000000180022cd8     libclrfmodw001.obj
 0003:0001ace0       ?inputPos@@3PEAEEA         0000000180022ce0     libclrfmodw001.obj
 0003:0001ace8       ?endPos@@3PEBEEB           0000000180022ce8     libclrfmodw001.obj
 0003:0001acf0       ?genPos@@3PEAEEA           0000000180022cf0     libclrfmodw001.obj
 0003:0001acf8       ?markPos@@3PEAEEA          0000000180022cf8     libclrfmodw001.obj
 0003:0001ad00       ?constantPool@@3PEAPEADEA  0000000180022d00     libclrfmodw001.obj
 0003:0001ad08       ?constantPoolCount@@3GA    0000000180022d08     libclrfmodw001.obj
 0003:0001ad0c       ?zeroBytes@@3PAEA          0000000180022d0c     libclrfmodw001.obj
 0003:0001ad10       ?codeLength@@3IA           0000000180022d10     libclrfmodw001.obj
 0003:0001ad14       result                     0000000180022d14     libclrfmodw001.obj
 0003:0001ad18       ?map@@3PEAIEA              0000000180022d18     libclrfmodw001.obj
 0003:0001ad20       ?widening@@3PEACEA         0000000180022d20     libclrfmodw001.obj
 0003:0001ad28       jvmti                      0000000180022d28     libclrfmodw001.obj
 0003:0001ad30       callbacks                  0000000180022d30     libclrfmodw001.obj
 0003:0001ae68       caps                       0000000180022e68     libclrfmodw001.obj
 0003:0001ae78       thrown_fid                 0000000180022e78     libclrfmodw001.obj
 0003:0001ae90       GS_ExceptionRecord         0000000180022e90     MSVCRT:gs_report.obj
 0003:0001af30       GS_ContextRecord           0000000180022f30     MSVCRT:gs_report.obj
 0003:0001b400       ?g_tss_cv@@3U_RTL_CONDITION_VARIABLE@@A 0000000180023400     MSVCRT:thread_safe_statics.obj
 0003:0001b408       ?g_tss_event@@3PEAXEA      0000000180023408     MSVCRT:thread_safe_statics.obj
 0003:0001b410       ?g_tss_mutex@@3U_RTL_CRITICAL_SECTION@@A 0000000180023410     MSVCRT:thread_safe_statics.obj
 0003:0001b438       ?g_sleep_condition_variable_cs@@3P6AHPEAU_RTL_CONDITION_VARIABLE@@PEAU_RTL_CRITICAL_SECTION@@K@ZEA 0000000180023438     MSVCRT:thread_safe_statics.obj
 0003:0001b440       ?g_wake_all_condition_variable@@3P6AXPEAU_RTL_CONDITION_VARIABLE@@@ZEA 0000000180023440     MSVCRT:thread_safe_statics.obj
 0003:0001b44c       ?__proc_attached@@3HA      000000018002344c     MSVCRT:dll_dllmain.obj
 0003:0001b460       ?is_initialized_as_dll@@3_NA 0000000180023460     MSVCRT:utility.obj
 0003:0001b461       ?module_local_atexit_table_initialized@@3_NA 0000000180023461     MSVCRT:utility.obj
 0003:0001b468       ?module_local_atexit_table@@3U_onexit_table_t@@A 0000000180023468     MSVCRT:utility.obj
 0003:0001b480       ?module_local_at_quick_exit_table@@3U_onexit_table_t@@A 0000000180023480     MSVCRT:utility.obj
